:100000000C9482000C94AA000C94AA000C94AA00F0
:100010000C94AA000C94AA000C94AA000C94AA00B8
:100020000C94AA000C94AA000C94AA000C94AA00A8
:100030000C94AA000C94AA000C94AA000C94AA0098
:100040000C94B4120C94AA000C948C0F0C94DA0F3C
:100050000C94AA000C94AA000C94AA000C94AA0078
:100060000C94AA000C94AA000000000024002700B1
:100070002A0000000000250028002B0000000000DE
:1000800023002600290004040404040404040202DA
:100090000202020203030303030301020408102007
:1000A0004080010204081020010204081020000012
:1000B0000007000201000003040600000000000029
:1000C0000000494E46494E4954594E414ECDCCCC84
:1000D0003D0AD7233C17B7D13877CC2B329595E61C
:1000E000241FB14F0A000020410000C84200401CFC
:1000F0004620BCBE4CCA1B0E5AAEC59D74004407B8
:1001000046113D0711241FBECFEFD8E0DEBFCDBFA3
:1001100011E0A0E0B1E0ECEAF1E302C005900D923D
:10012000AE3EB107D9F713E0AEEEB1E001C01D92CB
:10013000A530B107E1F710E0C2E0D1E004C022979A
:10014000FE010E948318CE3FD107C9F70E949C117F
:100150000C94C9180C940000CF93DF93BC0182303B
:10016000910510F462E070E0A0910103B0910203E8
:10017000ED01E0E0F0E040E050E021C088819981AD
:100180008617970769F48A819B81309719F09383CA
:10019000828304C09093020380930103FE0134C064
:1001A0006817790738F44115510519F08417950738
:1001B00008F4AC01FE018A819B819C01E901209732
:1001C000E9F641155105A9F1CA01861B970B049761
:1001D00008F4BA01E0E0F0E02AC08D919C911197FB
:1001E00084179507F9F46417750781F412968D91B9
:1001F0009C911397309719F09383828304C0909356
:10020000020380930103FD0132964CC0CA01861B94
:10021000970BFD01E80FF91F6193719302978D937E
:100220009C9340C0FD01828193819C01D90110976C
:10023000A1F68091FF0290910003892B41F48091F7
:10024000C9019091CA01909300038093FF024091ED
:10025000CB015091CC014115510541F44DB75EB72A
:100260008091C7019091C801481B590B2091FF0252
:1002700030910003CA01821B930B8617970780F009
:10028000AB014E5F5F4F8417950750F0420F531F2D
:10029000509300034093FF02F9016193719302C0F0
:1002A000E0E0F0E0CF01DF91CF910895CF93DF93AD
:1002B000009709F450C0EC0122971B821A82A0918A
:1002C0000103B0910203109709F140E050E0AC1730
:1002D000BD0708F1BB83AA83FE0121913191E20F92
:1002E000F31FAE17BF0779F48D919C911197280FDA
:1002F000391F2E5F3F4F3983288312968D919C9131
:1003000013979B838A834115510571F4D09302039F
:10031000C093010320C012968D919C911397AD015B
:10032000009711F0DC01D3CFFA01D383C28321916E
:100330003191E20FF31FCE17DF0769F488819981AD
:10034000280F391F2E5F3F4FFA01318320838A81A6
:100350009B8193838283DF91CF910895A0E0B0E0E9
:10036000E4EBF1E00C9494186C01009729F4CB01B4
:100370000E94AC006C01C1C08EEF882E8FEF982ECA
:100380008C0C9D1C8601060F171F0815190508F413
:10039000B2C0F401A081B181A617B707B8F0A530AB
:1003A000B10508F4AAC0CD0104978617970708F491
:1003B000A4C01297A61BB70BF801A193B193D40167
:1003C0006D937C93CF010E94560197C07B01EA1A7E
:1003D000FB0AEEEFFFEFEE0EFF1E36016A0E7B1EEC
:1003E000C0910103D091020344245524AA24BB24C4
:1003F0004AC0C615D705E1F5488159814E155F05FC
:10040000B8F1CA0104978E159F05B0F41296A40F97
:10041000B51FF401B183A0832A813B8141145104AB
:1004200031F0D20113963C932E93129766C030930D
:1004300002032093010361C08A819B81F8019383A9
:100440008283425050404E195F09518340834114CA
:10045000510431F0D20113961C930E93129704C0ED
:100460001093020300930103F4017183608345C07C
:1004700088819981A816B90608F45C012E018A8149
:100480009B819C01E901209709F0B3CF8091FF0285
:100490009091000386159705E9F4A616B706D0F4E7
:1004A0002091CB013091CC012115310541F42DB7BC
:1004B0003EB78091C7019091C801281B390B0217E4
:1004C0001307C8F4109300030093FF02D4016D9347
:1004D0007C9313C0CB010E94AC00EC01009759F053
:1004E000F40140815181B6010E948702C6010E9439
:1004F00056016E0102C0CC24DD24C601CDB7DEB7A3
:10050000E0E10C94B018662777270C94D504FB0122
:10051000DC0102C001900D9241505040D8F708957F
:10052000FC018191861721F08823D9F79927089536
:100530003197CF010895FB01DC018D910190801965
:100540000110D9F3990B0895FB01DC0101900D9284
:100550000020E1F70895FB01DC014150504048F0D4
:1005600001900D920020C9F701C01D9241505040EA
:10057000E0F70895FB0151915523A9F0BF01DC017B
:100580004D9145174111E1F759F4CD01019000203B
:1005900049F04D9140154111C9F3FB014111EFCFD5
:1005A00081E090E001970895AEE0B0E0EAEDF2E07E
:1005B0000C94A0180D891E8986E08C831A83098308
:1005C0008FEF9FE79E838D839E01275E3F4FCE0175
:1005D00001966F89788DA9010E94F8022F813885D4
:1005E000020F131FF80110822E96E4E00C94BC1841
:1005F000ABE0B0E0EEEFF2E00C9492183C012B017E
:100600005A01FC0117821682838181FD03C06FEFBE
:100610007FEFC6C19AE0892E1E010894211C311C6F
:10062000F3012381F20123FD859123FF81912F01A5
:10063000882309F4B2C1853239F423FD859123FF63
:1006400081912F01853229F490E0B3010E94630665
:10065000E7CF982FFF24EE249924FFE1FF15D0F077
:100660009B3269F09C3228F4903259F0933291F425
:100670000EC09D3249F0903369F441E024C052E04D
:10068000F52A84E0F82A28C098E0F92A25C0E0E19C
:10069000FE2A22C0F7FC29C0892F80538A3070F4CB
:1006A000F6FE05C0989C902C1124980E15C0E89C6D
:1006B000E02C1124E80EF0E2FF2A0EC09E3229F44D
:1006C000F6FC6BC140E4F42A07C09C3619F450E8EC
:1006D000F52A02C0983649F4F20123FD959123FFD3
:1006E00091912F01992309F0B8CF892F8554833038
:1006F00018F08052833038F444E050E0A40EB51E68
:100700005FE359830FC0933631F0933779F0933517
:1007100009F056C020C0F5018081898342E050E095
:10072000A40EB51E610101E010E012C0F501C08009
:10073000D180F6FC03C06FEF7FEF02C0692D70E03F
:1007400042E050E0A40EB51EC6010E9458068C017E
:100750005FE7F52214C0F501C080D180F6FC03C02C
:100760006FEF7FEF02C0692D70E042E050E0A40E11
:10077000B51EC6010E944D068C0150E8F52AF3FE15
:1007800007C01AC080E290E0B3010E946306EA94B9
:100790008E2D90E008171907A8F30EC0F601F7FC9C
:1007A0008591F7FE81916F0190E0B3010E9463068D
:1007B000E110EA94015010400115110579F7EAC0E3
:1007C000943611F0993669F5F7FE08C0F5012081DD
:1007D00031814281538184E090E00AC0F50180813B
:1007E00091819C01442737FD4095542F82E090E091
:1007F000A80EB91E9FE6F92257FF09C050954095F3
:10080000309521953F4F4F4F5F4FE0E8FE2ACA01D8
:10081000B901A1012AE030E00E948F06D82ED2183B
:1008200040C0953729F41F2D1F7E2AE030E01DC0FF
:100830001F2D197F9F3661F0903720F4983509F00D
:10084000ACC00FC0903739F0983709F0A6C004C08B
:1008500028E030E00AC0106114FD146020E130E0AF
:1008600004C014FD166020E132E017FF08C0F50156
:10087000608171818281938144E050E008C0F5017C
:1008800080819181BC0180E090E042E050E0A40EC4
:10089000B51EA1010E948F06D82ED2188FE7F82E20
:1008A000F122F6FE0BC05EEFF522D91438F4F4FE07
:1008B00007C0F2FC05C08FEEF82202C01D2D01C05A
:1008C000192DF4FE0DC0FE01ED0DF11D8081803368
:1008D00019F499EEF92208C01F5FF2FE05C003C0AB
:1008E0008F2D867809F01F5F0F2DF3FC14C0F0FEEA
:1008F0000FC01E1510F09D2C0BC09D2C9E0C911A44
:100900001E2D06C080E290E0B3010E9463061F5FC7
:100910001E15C0F304C01E1510F4E11A01C0EE2428
:1009200004FF0FC080E390E0B3010E94630602FF62
:100930001DC001FD03C088E790E00EC088E590E08F
:100940000BC0802F867891F001FF02C08BE201C0BE
:1009500080E2F7FC8DE290E0B3010E94630606C0DE
:1009600080E390E0B3010E9463069A94D914C0F327
:10097000DA94F101ED0DF11D808190E0B3010E9448
:100980006306DD20A9F706C080E290E0B3010E9473
:100990006306EA94EE20C1F743CEF30166817781C6
:1009A000CB012B96E2E10C94AE18A0E0B0E0EBEDA9
:1009B000F4E00C949818EC015B016115710519F0D5
:1009C000FB0191838083F9908F2D90E00E9487181E
:1009D000892BC9F7FDE2FF1621F4F990EE24E39488
:1009E00005C02BE2F21609F4F990EE248E010150B5
:1009F0001040C80162EC70E043E050E00E94350610
:100A0000892B01F58E010E5F1F4FC80165EC70E068
:100A100045E050E00E943506892B19F48E01095FEC
:100A20001F4FA114B10419F0F50111830083E0FCFC
:100A300004C070E090E080E814C070E090E080E8CE
:100A40006FEF08C1C8016AEC70E043E050E00E941B
:100A50003506892B69F4A114B10429F470E090E003
:100A600080EC6FE7F7C02296F501D183C083F6CF03
:100A70008824992440E050E060E070E0EF2DE053DE
:100A8000EA30A0F5F2E0EF2A8E2D90E09C0128706C
:100A90003070E2FE06C0232B79F50894811C911C6E
:100AA0002BC0232B19F0089481089108DB01CA019F
:100AB00012E0880F991FAA1FBB1F1A95D1F7480F84
:100AC000591F6A1F7B1F440F551F661F771F4E0F4C
:100AD000511D611D711D483929E9520729E9620735
:100AE00029E1720748F084E0E82A06C0EE3F31F4BD
:100AF000E3FC39C098E0E92AF990C0CFE53311F062
:100B0000E53189F529912D3219F4E0E1EE2A05C08D
:100B10002B3219F081E090E003C0299182E090E04F
:100B2000E22FE053EA3018F0C81BD90B1CC020E0BC
:100B300030E0FCE020383F075CF4C901880F991FC2
:100B4000880F991F280F391F220F331F2E0F311DB9
:100B5000E991E053EA3068F3E4FE03C03095219553
:100B60003F4F820E931ECE2CDD24E1FE07C0A11460
:100B7000B10421F02197F501D183C083CB01BA01E3
:100B80000E9404177B018C01F3E0CF22DD2423E0D7
:100B9000C216D10421F417FB109517F910955701CF
:100BA0006801C801B70120E030E040E050E00E9459
:100BB000CF16882309F44AC097FE0DC021EEE22E1D
:100BC00020E0F22E9094819491089394C0E2D0E0BA
:100BD00000E010E012C099EFE92E90E0F92EF6CF78
:100BE000F7012591359145915491C601B5010E94B7
:100BF000BA175B016C018C1A9D0A8C169D0684F74E
:100C0000D595C7950F5F1F4F0630110529F08CEF62
:100C10009FEFE80EF91EF1CFC501D6017C018D01D1
:100C20008C2D880F8D2D881F8F3F51F0C601B50187
:100C300020E030E040E050E00E94CF16882331F4FD
:100C400082E290E090930403809303037E2D9F2D16
:100C5000802F612F272F392F482F562FB901CA0116
:100C6000CDB7DEB7ECE00C94B418FB01DC014150C9
:100C7000504088F08D9181341CF08B350CF4805EEF
:100C8000659161341CF06B350CF4605E861B61115C
:100C900071F3990B0895881BFCCFFC0105906150FE
:100CA00070400110D8F7809590958E0F9F1F089582
:100CB000FC016150704001900110D8F7809590952B
:100CC0008E0F9F1F08950F931F93CF93DF938C0177
:100CD000EB018B8181FF1BC082FF0DC02E813F8104
:100CE0008C819D812817390764F4E881F98101938B
:100CF000F983E88306C0E885F985802F0995892B5B
:100D000031F48E819F8101969F838E8302C00FEF05
:100D10001FEFC801DF91CF911F910F910895FA0144
:100D2000AA27283051F1203181F1E8946F936E7F2A
:100D30006E5F7F4F8F4F9F4FAF4FB1E03ED0B4E01B
:100D40003CD0670F781F891F9A1FA11D680F791F5C
:100D50008A1F911DA11D6A0F711D811D911DA11D6D
:100D600020D009F468943F912AE0269F112430197D
:100D7000305D3193DEF6CF010895462F4770405D18
:100D80004193B3E00FD0C9F7F6CF462F4F70405DC7
:100D90004A3318F0495D31FD4052419302D0A9F722
:100DA000EACFB4E0A6959795879577956795BA951C
:100DB000C9F700976105710508959B01AC010A2EE2
:100DC00006945795479537952795BA95C9F7620FB9
:100DD000731F841F951FA01D0895EF92FF920F931C
:100DE0001F938130910551F0892B19F46F5F7F4F6C
:100DF000A1F11F910F91FF90EF9008956F5F7F4FCA
:100E0000C1F70EEE11E0C80160E071E00E94AB1581
:100E1000095F1F4F82E00A301807A9F785E192E0C9
:100E200068EC70E048E050E029E030E00AE010E0D3
:100E3000FBE0EF2EF12C0E94500F8FE292E068EC65
:100E400070E042E050E023E030E004E010E0E5E054
:100E5000EE2EF12C0E94500FCCCF03E012E0C8011F
:100E60000E945E160750104081E0073E1807B9F750
:100E70001F910F91FF90EF90089580E090E06FEF49
:100E80007FEF0E94ED06089581E090E06FEF7FEF25
:100E90000E94ED0608950F931F93DF93CF93CDB774
:100EA000DEB7C45FD1400FB6F894DEBF0FBECDBF32
:100EB0008DB79EB70C970FB6F8949EBF0FBE8DBF2F
:100EC000EDB7FEB731968E010F5F1F4FADB7BEB7BE
:100ED00012961C930E93119781E091E09383828385
:100EE00087E391E09583848381E090E09783868314
:100EF0008FEF9FEF9187808784E190E093878287CF
:100F00000E94D4028DB79EB70C960FB6F8949EBF80
:100F10000FBE8DBF83ED92E0B8010E941112CC503C
:100F2000DE4F0FB6F894DEBF0FBECDBFCF91DF917D
:100F30001F910F9108950F931F93DF93CF93CDB718
:100F4000DEB7E2970FB6F894DEBF0FBECDBF8DB708
:100F50009EB70C970FB6F8949EBF0FBE8DBFEDB72E
:100F6000FEB731968E010F5F1F4FADB7BEB7129619
:100F70001C930E93119780E591E093838283809177
:100F8000D5019091D601A091D701B091D801848369
:100F90009583A683B7838091D9019091DA01A091BE
:100FA000DB01B091DC0180879187A287B3870E9423
:100FB000D4028DB79EB70C960FB6F8949EBF0FBEA5
:100FC0008DBF83ED92E0B8010E941112E2960FB638
:100FD000F894DEBF0FBECDBFCF91DF911F910F916F
:100FE000089583ED92E06AE571E00E941112089580
:100FF000BC0183ED92E00E94571208950F931F9356
:10100000DF93CF93CDB7DEB727970FB6F894DEBF47
:101010000FBECDBF81E0809314028E010F5F1F4F82
:10102000C80166E671E00E94AB15C8010E94F8078E
:10103000C8010E945E1627960FB6F894DEBF0FBE59
:10104000CDBFCF91DF911F910F9108950F931F9303
:10105000DF93CF93CDB7DEB727970FB6F894DEBFF7
:101060000FBECDBF109214028E010F5F1F4FC8013B
:1010700066E671E00E94AB15C8010E94F807C8013E
:101080000E945E1627960FB6F894DEBF0FBECDBF46
:10109000CF91DF911F910F9108950F931F93DF93CD
:1010A000CF93CDB7DEB727970FB6F894DEBF0FBE4C
:1010B000CDBF1092CD011092CE011092CF011092AF
:1010C000D0011092D1011092D2011092D30110924E
:1010D000D4018E010F5F1F4FC80166E671E00E94C8
:1010E000AB15C8010E94F807C8010E945E1627963A
:1010F0000FB6F894DEBF0FBECDBFCF91DF911F9129
:101100000F9108950F931F93DF93CF93CDB7DEB761
:1011100027970FB6F894DEBF0FBECDBF0E94D8163A
:101120000E9430138E010F5F1F4FC80166E671E009
:101130000E94AB15C8010E94F807C8010E945E1604
:1011400027960FB6F894DEBF0FBECDBFCF91DF91CB
:101150001F910F910895FC01662349F4EE0FFF1FC4
:10116000E65FFD4F808160E00E94FD130895EE0F61
:10117000FF1FE65FFD4F808161E00E94FD1308952F
:101180000F931F93DF93CF93CDB7DEB727970FB69B
:10119000F894DEBF0FBECDBF8C01809112029091FA
:1011A0001302009701F5043011051CF1109213028F
:1011B000109212028E010F5F1F4FC80166E671E0A8
:1011C0000E94AB15C8010E94F807C8010E945E1674
:1011D00027960FB6F894DEBF0FBECDBFCF91DF913B
:1011E0001F910F91089561E00E94AB080430110532
:1011F000ECF6C80160E00E94AB0810931302009364
:101200001202D8CF2F923F924F925F926F927F92AD
:101210008F929F92AF92BF92CF92DF92EF92FF9206
:101220000F931F93DF93CF93CDB7DEB72C970FB6F5
:10123000F894DEBF0FBECDBF6B837C838D839E830E
:101240002F83388749875A8785E192E0B801A70143
:101250000E94500E8FE292E0B801A7010E94500E4A
:1012600080911402882361F16091CD017091CE01CB
:101270008091CF019091D0010E9404179B01AC0195
:101280006B817C818D819E810E946B166B837C8338
:101290008D839E836091D1017091D2018091D301A1
:1012A0009091D4010E9404179B01AC016F81788555
:1012B00089859A850E946B166F83788789879A87BC
:1012C0006B817C818D819E8120E030E040EA51E499
:1012D0000E94B61718160CF00CC180E090E0A0EA4E
:1012E000B1E48B839C83AD83BE8398EEE92E93E0BB
:1012F000F92E012D112D88EEC82E83E0D82E6F8196
:10130000788589859A8520E030E048E452E40E949F
:10131000BA170E94D3162091CD013091CE01409191
:10132000CF015091D0012E153F054007510709F418
:101330002EC15601A21AB30ACB01AA2797FDA09588
:10134000BA2FE090D101F090D2010091D301109119
:10135000D4018E159F05A007B10709F414C16B01D4
:10136000CE18DF08CA01B9010E9404179B01AC0125
:101370006B817C818D819E810E94B61718160CF4BA
:10138000B3C0AFEFBFEFBA83A983C801B7010E9412
:1013900004179B01AC016F81788589859A850E942D
:1013A000B61718160CF49BC08FEF9FEF9C878B87A6
:1013B000CA14DB040CF441C03601882477FC809405
:1013C000982C611471048104910409F441C0150141
:1013D000442437FC4094542CEE24FF248701AA2493
:1013E000BB24650110C060E070E080E090E00E94E6
:1013F00030130894A11CB11CC11CD11CA614B70445
:10140000C804D90428F58FE292E06B857C850E94A0
:10141000EE0EE20CF31C041D151DE614F70408057E
:10142000190508F3E618F7080809190985E192E09B
:1014300069817A810E94EE0ED6CF3501882477FC2F
:101440008094982C611471048104910409F064C0A3
:101450006B817C818D819E810E94D8167B018C01DD
:101460006093CD017093CE018093CF019093D00112
:101470006F81788589859A850E94D8166093D101FD
:101480007093D2018093D3019093D401E092D5015F
:10149000F092D6010093D7011093D8016093D9013F
:1014A0007093DA018093DB019093DC012C960FB6E8
:1014B000F894DEBF0FBECDBFCF91DF911F910F918A
:1014C000FF90EF90DF90CF90BF90AF909F908F9064
:1014D0007F906F905F904F903F902F900895A1E084
:1014E000B0E0BC87AB8764CFE1E0F0E0FA83E9834A
:1014F0004CCF6B817C818D819E8120E030E048E47F
:1015000052E40E94BA170E94D3167B010027F7FC11
:101510000095102F6B01F3CE1601442437FC409444
:10152000542CEE24FF248701AA24BB24650111C09A
:1015300060E070E080E090E00E9430130894A11C0D
:10154000B11CC11CD11CA614B704C804D90408F0EE
:101550007FCF85E192E069817A810E94EE0EE20CF4
:10156000F31C041D151DE614F7040805190500F306
:10157000E618F708080919098FE292E06B857C8567
:101580000E94EE0ED5CF6701C61AD70AEBCE5701DF
:10159000AC18BD08D1CEEF92FF920F931F93DF934B
:1015A000CF93CDB7DEB727970FB6F894DEBF0FBE47
:1015B000CDBFF6E9EF2EF12C012D112D0E9402096D
:1015C0008E010F5F1F4FC80166E671E00E94AB15E8
:1015D000C8010E94F807C8010E945E1627960FB640
:1015E000F894DEBF0FBECDBFCF91DF911F910F9159
:1015F000FF90EF900895CF92DF92EF92FF920F93BA
:101600001F93DF93CF93CDB7DEB727970FB6F8942C
:10161000DEBF0FBECDBFD82EC92E7B018E010F5F5E
:101620001F4FC80169E671E00E94AB15C701B80100
:101630000E9474149C018D2D9C2DB70140E050E058
:101640000E94DE15C8010E945E168D2D9C2D2796E6
:101650000FB6F894DEBF0FBECDBFCF91DF911F91C3
:101660000F91FF90EF90DF90CF900895AF92BF92CF
:10167000CF92DF92EF92FF920F931F93DF93CF935E
:10168000CDB7DEB7C054D0400FB6F894DEBF0FBE62
:10169000CDBF7C01162F0E9497146C015E01089447
:1016A000A11CB11CC50169E671E00E94AB15C70120
:1016B000612F0E949714AC01C701B5010E94561416
:1016C0009C018E01085F1F4F0894C11CD11CC801EA
:1016D000B701A6010E94DE15AFE0EA2EF12CEC0E58
:1016E000FD1EC801B70142E350E020E030E00E9457
:1016F0009C14C8010E945E16C5010E945E16C701B7
:101700000E948302C05CDF4F0FB6F894DEBF0FBEAD
:10171000CDBFCF91DF911F910F91FF90EF90DF90A0
:10172000CF90BF90AF9008954F925F926F927F924B
:101730008F929F92AF92BF92CF92DF92EF92FF92E1
:101740000F931F93DF93CF93CDB7DEB7E8970FB614
:10175000F894DEBF0FBECDBF582E492E3B018E013F
:101760000F5F1F4FC8016BE671E00E94AB15C3010C
:10177000B8010E9474147C01C8010E945E168FEFAC
:10178000E8168FEFF80681F18E01085F1F4FC80140
:101790006BE671E00E94AB15C301B8010E9474149E
:1017A0009C01852D942DB30140E050E00E94DE1590
:1017B000C8010E945E16852D942DE8960FB6F89408
:1017C000DEBF0FBECDBFCF91DF911F910F91FF9074
:1017D000EF90DF90CF90BF90AF909F908F907F90D1
:1017E0006F905F904F9008958E01015F1F4FC80169
:1017F0006DE671E00E94AB15C301B8010E9474143C
:101800007C01C8010E945E168FEFE8168FEFF80684
:1018100009F452C086E1882E912C8C0E9D1EC401C5
:101820006DE671E00E94AB15C301B4010E9474140F
:101830009C010DE1A02EB12CAC0EBD1EC501B30163
:1018400040E050E00E94DE1512E3C12ED12CCC0EF8
:10185000DD1EC601B5010E945316B4E2EB2EF12C39
:10186000EC0EFD1EC7016FE671E00E94AB15C301CF
:10187000B7010E947414AC018E01055D1F4FC801B1
:10188000B3010E942516C601B8010E947415BC015F
:10189000852D942D0E944816C8010E945E16C7012E
:1018A0000E945E16C6010E946416C5010E945E1663
:1018B000C4010E945E167FCF852D942DB3010E9436
:1018C000481679CF6F927F928F929F92AF92BF927C
:1018D000CF92DF92EF92FF920F931F93DF93CF93FC
:1018E000CDB7DEB7CB55D0400FB6F894DEBF0FBEF4
:1018F000CDBF4C017E010894E11CF11CC701B4016D
:101900000E9448168E01085F1F4FC801B7010E9450
:10191000940BC401B8010E943116C8010E945E16E2
:10192000C7010E945E168E010A5E1F4FC801B401F6
:101930000E9448165FE0652E712C6C0E7D1EC3015F
:10194000B8010E94FB0AC8010E945E16C40160E053
:1019500070E00E943014FC010081C30161E771E076
:101960000E94C914882309F083C0C30164E771E0B1
:101970000E94C9148823E9F5C30167E771E00E945A
:10198000C914882309F087C0C3016AE771E00E9487
:10199000C914882309F090C0C3016EE771E00E946A
:1019A000C914882309F08BC0C30162E871E00E946A
:1019B000C914882309F086C0C30166E871E00E945B
:1019C000C914882309F481C08E01005C1F4FC8012F
:1019D000B4010E944816C80164E50E94360B0E94BB
:1019E000D316DC01CB010E94C008C8010E945E161C
:1019F00026C03BE2A32EB12CAC0EBD1EC501B40126
:101A00000E944816C50168E50E94360B6B017C01F7
:101A10008E010E5C1F4FC801B4010E944816C80118
:101A200069E50E94360B9B01AC01C701B6010E941B
:101A3000CB0AC8010E945E16C5010E945E16C30152
:101A40000E945E16C55ADF4F0FB6F894DEBF0FBE78
:101A5000CDBFCF91DF911F910F91FF90EF90DF905D
:101A6000CF90BF90AF909F908F907F906F90089590
:101A70004DE1A42EB12CAC0EBD1EC501B4010E94D7
:101A80004816C50168E50E94360B6B017C018E018A
:101A90000C5D1F4FC0CF8E01075C1F4FC801B40102
:101AA0000E944816C80160E50E94360B0E94820819
:101AB000C8010E945E16C3CF0E944D08C0CF0E948D
:101AC0002608BDCF0E94FE07BACF043509F47CCFAB
:101AD000C30163EB71E00E94C914882359F5C30167
:101AE00068E871E00E94C914882339F5C3016DE8E4
:101AF00071E00E94C914882331F5C30162E971E0E5
:101B00000E94C914882311F5C30167E971E00E949E
:101B1000C9148823F1F48E010B5A1F4FC8016CE9D8
:101B200071E00E94AB15C8010E94F807C8010E942D
:101B30005E1685CF0E94F10782CFE0914902F091B5
:101B40004A0209957CCF0E949B0779CF0E944B07E0
:101B500076CF8E01095B1F4FC80167E971E00E94D3
:101B6000AB15C401B8010E9474142EE4E22EF12CCE
:101B7000EC0EFD1EAC014C5F5F4FC701B4010E942B
:101B80002516C7010E94F807C7010E945E16C8010A
:101B90000E945E1654CFEF92FF920F931F93DF9334
:101BA000CF93CDB7DEB72E970FB6F894DEBF0FBE3A
:101BB000CDBF83ED92E00E949C10892BC9F07E017D
:101BC0000894E11CF11CC70163ED72E00E949712BA
:101BD0008E01085F1F4FC801B7010E944816C80157
:101BE0000E94620CC8010E945E16C7010E945E1628
:101BF0002E960FB6F894DEBF0FBECDBFCF91DF910A
:101C00001F910F91FF90EF900895CF93DF93CCE059
:101C1000D2E0888161E00E949113888161E00E9496
:101C2000FD13229682E0C231D80799F7DF91CF9158
:101C300008950F931F9305EF11E0C80166EB71E063
:101C40000E94C515C80107966BEB71E00E94C5158F
:101C5000C8010E9660EC71E00E94C5151F910F91AE
:101C6000089583ED92E040E855E260E070E00E9464
:101C700015100E94050E0E94190E86E090E09093C8
:101C80000D0280930C0287E090E090930F02809306
:101C90000E028CE090E09093110280931002089560
:101CA000CF92DF92EF92FF920F931F936C017A0114
:101CB0008B01FC0120853185442737FD4095542F49
:101CC00060E67AEE80E090E00E945218CA01B90105
:101CD000A80197010E945218F60124833583468398
:101CE00057831F910F91FF90EF90DF90CF90089551
:101CF0000F931F93CF93DF93EC018B018A859B8514
:101D0000029731F56130710589F06230710524F474
:101D10006115710541F01CC06230710571F06330CE
:101D20007105B1F40DC08E8560E002C08E8561E062
:101D30000E94FD13888961E009C08E8561E002C0C0
:101D40008E8560E00E94FD13888960E00E94FD138B
:101D50008A859B850497E9F501301105A1F00230D1
:101D600011051CF4012B41F034C002301105D1F0F3
:101D70000330110571F51DC08E8561E00E94FD13D1
:101D8000888960E006C08E8560E00E94FD13888926
:101D900061E00E94FD138A8961E00E94FD138C8935
:101DA00060E015C08E8560E00E94FD13888961E0C7
:101DB00006C08E8561E00E94FD13888960E00E9464
:101DC000FD138A8960E00E94FD138C8961E00E9406
:101DD000FD13DF91CF911F910F9108950F931F93E2
:101DE000CF93DF93EC011616170624F481E090E000
:101DF0009983888377FF02C0198218828B0177FF4D
:101E000046C0109501951F4F42C00E94FC122E89BA
:101E10003F89488D598D621B730B840B950B2C8168
:101E20003D814E815F81621773078407950768F3D0
:101E30000E94FC126E8B7F8B888F998F888199818D
:101E40002C853D85019761F42F5F3F4F3D872C879F
:101E5000888599852817390771F41D861C860BC063
:101E6000232B21F4888599859D878C878C859D857A
:101E700001979D878C87015010408C859D8564E07B
:101E800070E00E941D18BC01CE010E94780E011561
:101E9000110509F0BACFDF91CF911F910F910895ED
:101EA000CF92DF92EF92FF920F931F936C01842FDA
:101EB000F601158614861382128211821082168A08
:101EC000178A108E118E7187608746875787318BEE
:101ED000208B138B028BF58AE48A61E00E949113B8
:101EE000F601808961E00E949113F601828961E028
:101EF0000E949113F601848961E00E94911384E0AD
:101F000090E0F601938782871F910F91FF90EF90E9
:101F1000DF90CF90089508951F920F920FB60F9201
:101F200011242F933F934F938F939F93EF93FF939E
:101F30008091C00082FD1DC04091C60020918B029F
:101F400030918C022F5F3F4F2F73307080918D0244
:101F500090918E022817390771F0E0918B02F09171
:101F60008C02E55BFD4F408330938C0220938B0203
:101F700002C08091C600FF91EF919F918F914F9188
:101F80003F912F910F900FBE0F901F901895E091E9
:101F9000DF02F091E002E05CFF4F8191919120819E
:101FA0003181821B930B8F739070892B11F00E94EB
:101FB0008B0F08951F920F920FB60F9211242F933B
:101FC0003F938F939F93EF93FF932091CF02309194
:101FD000D0028091D1029091D2022817390731F4B2
:101FE0008091C1008F7D8093C10014C0E091D10227
:101FF000F091D202E157FD4F20818091D102909162
:10200000D20201968F7390709093D2028093D10286
:102010002093C600FF91EF919F918F913F912F9157
:102020000F900FBE0F901F901895AF92BF92DF9246
:10203000EF92FF920F931F93CF93DF93EC017A01FE
:102040008B01DD24403081EE580780E0680780E096
:10205000780711F0DD24D39491E0A92EB12CEC89FE
:10206000FD89DD2069F0C50108A002C0880F991F15
:102070000A94E2F7808360E079E08DE390E005C0A8
:10208000108260E874E88EE190E0A80197010E9458
:102090003018215030404040504056954795379574
:1020A000279580E12030380720F0DD2011F0DD2475
:1020B000D6CFE889F9893083EA89FB89208319A280
:1020C000EE89FF89408121E030E0C9010C8C02C01B
:1020D000880F991F0A94E2F7482B4083EE89FF8905
:1020E0004081C9010D8C02C0880F991F0A94E2F744
:1020F000482B4083EE89FF894081C9010E8C02C0C4
:10210000880F991F0A94E2F7482B4083EE89FF89D4
:1021100080810F8C02C0220F331F0A94E2F72095B2
:1021200028232083DF91CF911F910F91FF90EF9093
:10213000DF90BF90AF900895DC011C96ED91FC916B
:102140001D97E05CFF4F2191319180819181281B87
:10215000390B2F733070C9010895DC011C96ED9185
:10216000FC911D97E05CFF4F20813181E054F040ED
:10217000DF01AE5BBF4F8D919C91119728173907F6
:1021800019F42FEF3FEF07C08D919C91E80FF91FD5
:102190008081282F30E0C9010895DC011C96ED9163
:1021A000FC911D97E05CFF4F20813181E054F040AD
:1021B000DF01AE5BBF4F8D919C91119728173907B6
:1021C00019F42FEF3FEF10C08D919C911197E80FFC
:1021D000F91F20818D919C91119701968F739070BA
:1021E00011969C938E9330E0C9010895DC0191967D
:1021F0008C919197882339F05496ED91FC915597E5
:10220000808186FFF9CF91961C920895CF93DF933A
:10221000EC01EE85FF85E05CFF4F20813181E054C9
:10222000F0402F5F3F4F2F733070DF01AE5BBF4F29
:102230008D919C91119728173907D1F3E05CFF4FDE
:1022400080819181E054F040E80FF91F6083EE85B2
:10225000FF85E05CFF4F31832083EE89FF89208179
:1022600081E090E00F8C02C0880F991F0A94E2F77A
:10227000282B208381E089A3EC89FD8980818064FB
:10228000808381E090E0DF91CF9108951092D60293
:102290001092D50288EE93E0A0E0B0E08093D702E0
:1022A0009093D802A093D902B093DA0281EE91E024
:1022B0009093D4028093D3028BE492E09093E00257
:1022C0008093DF028FE892E09093E2028093E10234
:1022D00085EC90E09093E4028093E30284EC90E03C
:1022E0009093E6028093E50280EC90E09093E80200
:1022F0008093E70281EC90E09093EA028093E902F8
:1023000082EC90E09093EC028093EB0286EC90E0FC
:102310009093EE028093ED0284E08093EF0283E0DD
:102320008093F00287E08093F10285E08093F202CF
:1023300081E08093F3020895CF93DF930E945613B8
:102340000E94310EC7ECDFE00E94CB0D2097E1F335
:102350000E94C70FF9CFCF92DF92EF92FF920F93B7
:102360001F93CF93DF937C016B018A01C0E0D0E023
:102370000FC0D6016D916D01D701ED91FC910190D7
:10238000F081E02DC7010995C80FD91F01501040F9
:102390000115110571F7CE01DF91CF911F910F91BA
:1023A000FF90EF90DF90CF900895EF92FF920F9300
:1023B0001F938C01DC01ED91FC910190F081E02DE7
:1023C0006DE009957C01D801ED91FC910190F081BF
:1023D000E02DC8016AE009959C012E0D3F1DC90141
:1023E0001F910F91FF90EF900895CF93DF93EC0131
:1023F0006115710519F420E030E00FC0DB010D908C
:102400000020E9F71197A61BB70BE881F98102803C
:10241000F381E02DAD0109959C01C901DF91CF91B8
:102420000895EF92FF920F931F937C010E94F51184
:102430008C01C7010E94D511080F191FC8011F91F7
:102440000F91FF90EF900895AF92BF92CF92DF92DD
:10245000EF92FF920F931F93CF93DF935C016B0179
:10246000EE24FF24C0E0D0E010C0D501ED91FC9136
:1024700000811181C601BE010E944514682FC5016B
:10248000F8010995E80EF91E2196F60184819581DF
:10249000C817D90750F3C701DF91CF911F910F9152
:1024A000FF90EF90DF90CF90BF90AF900895EF92A4
:1024B000FF920F931F937C010E9424128C01C7018D
:1024C0000E94D5119C01200F311FC9011F910F914E
:1024D000FF90EF900895CF93DF93EC010E94FC12E0
:1024E000688779878A879B87E881F9810680F781E9
:1024F000E02DCE0109959C0197FF15C00E94FC12AA
:10250000288539854A855B85621B730B840B950B87
:102510002C813D814E815F81621773078407950787
:1025200018F32FEF3FEFC901DF91CF9108950F937B
:102530001F93CF93DF93182F092FEB0165EC71E008
:102540000E94AB1504C0812F902F0E944F15CE0121
:102550000E946B12BC0197FFF6CF812F902FDF9165
:10256000CF911F910F9108951F920F920FB60F9266
:1025700011242F933F938F939F93AF93BF93809199
:10258000F9029091FA02A091FB02B091FC02309105
:10259000FD020196A11DB11D232F2D5F2D3720F0C7
:1025A0002D570196A11DB11D2093FD028093F902C4
:1025B0009093FA02A093FB02B093FC028091F50283
:1025C0009091F602A091F702B091F8020196A11D38
:1025D000B11D8093F5029093F602A093F702B09399
:1025E000F802BF91AF919F918F913F912F910F90E2
:1025F0000FBE0F901F9018958FB7F8942091F90295
:102600003091FA024091FB025091FC028FBFB90158
:10261000CA0108959FB7F8942091F5023091F6020F
:102620004091F7025091F80286B5A89B06C08F3FF3
:1026300021F02F5F3F4F4F4F5F4F9FBF542F432FCE
:10264000322F2227280F311D411D511D82E0220FFC
:10265000331F441F551F8A95D1F7B901CA01089548
:10266000EF92FF920F931F93CF93DF937B018C0127
:102670000E940A13EB010EC00E940A136C1B7D0B13
:10268000685E7340C8F30894E108F1080109110974
:10269000C851DC4FE114F1040105110569F7DF9120
:1026A000CF911F910F91FF90EF900895789484B58A
:1026B000826084BD84B5816084BD85B5826085BD3E
:1026C00085B5816085BDEEE6F0E080818160808324
:1026D000E1E8F0E010828081826080838081816007
:1026E0008083E0E8F0E0808181608083E1EBF0E0CE
:1026F000808184608083E0EBF0E080818160808372
:10270000EAE7F0E08081846080838081826080835A
:102710008081816080838081806880831092C10085
:102720000895CF93DF93482F50E0CA0186569F4FFC
:10273000FC0134914A575F4FFA018491882369F173
:1027400090E0880F991FFC01E859FF4FA591B491C3
:10275000FC01EE58FF4FC591D491662351F42FB779
:10276000F8948C91932F909589238C938881892359
:102770000BC0623061F42FB7F8948C91932F909531
:1027800089238C938881832B88832FBF06C09FB7B2
:10279000F8948C91832B8C939FBFDF91CF910895F8
:1027A000833071F0843028F48130A1F0823021F53B
:1027B00014C08630B1F08730D1F08430E9F404C021
:1027C000809180008F7703C0809180008F7D8093FF
:1027D0008000089584B58F7702C084B58F7D84BD55
:1027E00008958091B0008F778093B0000895809114
:1027F000B0008F7D8093B0000895FF920F931F93D8
:10280000F62E482F50E0CA0182559F4FFC012491BB
:10281000CA0186569F4FFC0114914A575F4FFA0137
:1028200004910023C9F0222319F0822F0E94D013B3
:10283000E02FF0E0EE0FFF1FEE58FF4FA591B4918F
:102840009FB7F894FF2021F48C911095812302C04A
:102850008C91812B8C939FBF1F910F91FF900895B6
:10286000FC019B01848195816817790728F46081B8
:1028700071816115710529F41092FE026EEF72E00C
:1028800002C0620F731FCB010895FC018481958102
:102890006817790748F40190F081E02D309721F016
:1028A000E60FF71F8081089580E00895CF93DF93AE
:1028B000FC01DB01848195814817590760F4C081D0
:1028C000D1816D917C91CE01840F951F0E94BA0237
:1028D0009C01009719F42FEF3FEF02C02C1B3D0B1A
:1028E000C901DF91CF91089540E050E00E94561455
:1028F0000895CF93DF93FC01848195814817590790
:1029000068F4C081D181772767FD7095CE01840F6F
:10291000951F0E9490029C01009719F42FEF3FEF42
:1029200002C02C1B3D0BC901DF91CF91089540E0FF
:1029300050E00E94791408950F931F93CF93DF9373
:10294000FC018B0141155105F9F061157105E1F0AC
:10295000848195812817390718F0FB01108214C073
:1029600041505040EC01C21BD30B4C175D0708F4DB
:10297000EA0160817181620F731FC801AE010E947C
:10298000AB02C00FD11F1882DF91CF911F910F9121
:102990000895DC01FB0114968D919C911597892B6C
:1029A00031F461157105A9F090E0808108C00D90A7
:1029B000BC91A02D6115710529F490E08C918823BC
:1029C00049F407C0CD010E949B029C0190E0232B9B
:1029D00009F491E0892F08950F931F93CF93DF930C
:1029E000EC018B016F5F7F4F888199810E94AE015E
:1029F000009711F480E005C0998388831B830A83C4
:102A000081E0DF91CF911F910F910895CF93DF93D4
:102A1000EC0188819981892B29F08A819B81861715
:102A2000970760F4CE010E94EC14882341F08C815A
:102A30009D81892B19F4E881F981108281E0DF9171
:102A4000CF910895EF92FF920F931F93CF93DF934F
:102A5000EC017B016C817D81E114F104C1F0411531
:102A6000510599F08A01060F171FB8010E9406153B
:102A7000882369F0888199812C813D81820F931F81
:102A8000B7010E94A4021D830C8381E001C080E095
:102A9000DF91CF911F910F91FF90EF900895DF93F9
:102AA000CF9300D0CDB7DEB769831A82BE016F5FC6
:102AB0007F4F41E050E00E9422150F900F90CF9180
:102AC000DF910895CF93DF93EC018881998100977E
:102AD00011F00E945601198218821D821C821B82ED
:102AE0001A82DF91CF9108950F931F93182F092F0A
:102AF000FB0160817181448155810E9422158823E8
:102B000021F4812F902F0E946215812F902F1F9109
:102B10000F910895EF92FF920F931F93CF93DF933E
:102B2000EC017B018A01BA010E940615882321F479
:102B3000CE010E94621507C01D830C838881998194
:102B4000B7010E94A402CE01DF91CF911F910F9196
:102B5000FF90EF900895CF93DF93EC0119821882D4
:102B60001B821A821D821C821E826115710551F022
:102B7000DB010D900020E9F71197A61BB70BAD0103
:102B80000E948A15DF91CF9108950F931F93182FFC
:102B9000092F6115710559F0DB010D900020E9F74F
:102BA0001197A61BB70BAD010E948A1502C00E94A7
:102BB0006215812F902F1F910F910895BF92CF9290
:102BC000DF92EF92FF920F931F93CF93DF93082F23
:102BD000B92E6B017A01E9012417350710F4EA01D7
:102BE0007901802F9B2D66EC71E00E94AB15D60118
:102BF00014968D919C9115978E159F05D0F08C178A
:102C00009D0708F4EC01D601ED91FC911197EC0FB2
:102C1000FD1F108110826D917C916E0D7F1D802FA4
:102C20009B2D0E94C515D601ED91FC91EC0FFD1F67
:102C30001083802F9B2DDF91CF911F910F91FF90DB
:102C4000EF90DF90CF90BF9008950F931F938C016A
:102C5000FB01248135810E94DE15C8011F910F916F
:102C60000895CF93DF93EC01FB018617970761F07E
:102C7000608171816115710529F0448155810E943F
:102C80008A1502C00E946215CE01DF91CF9108958E
:102C9000FC01118210821382128215821482168224
:102CA0000E9431160895FC01118210821382128253
:102CB0001582148216820E9431160895FC018081CB
:102CC00091810E9456010895FC01808191810E94AA
:102CD000560108955058BB27AA270ED00DC1FED02B
:102CE00030F003D120F031F49F3F11F41EF4F3C013
:102CF0000EF4E095E7FBE9C0E92F0FD180F3BA1796
:102D0000620773078407950718F071F49EF527C1D1
:102D10000EF4E0950B2EBA2FA02D0B01B9019001F6
:102D20000C01CA01A0011124FF27591B99F0593F3A
:102D300050F4503E68F11A16F040A22F232F342F82
:102D40004427585FF3CF469537952795A795F040D0
:102D50005395C9F77EF41F16BA0B620B730B840BE5
:102D6000BAF09150A1F0FF0FBB1F661F771F881F9D
:102D7000C2F70EC0BA0F621F731F841F48F48795F5
:102D800077956795B795F7959E3F08F0B3CF9395E4
:102D9000880F08F09927EE0F97958795089571D0C1
:102DA00008F481E0089504D06894B111D9C0089561
:102DB000BCD088F09F5790F0B92F9927B751A0F059
:102DC000D1F0660F771F881F991F1AF0BA95C9F7BF
:102DD00012C0B13081F0C3D0B1E00895C0C0672FF8
:102DE000782F8827B85F39F0B93FCCF3869577956F
:102DF0006795B395D9F73EF4909580957095619558
:102E00007F4F8F4F9F4F0895E89409C097FB3EF482
:102E100090958095709561957F4F8F4F9F4F992327
:102E2000A9F0F92F96E9BB279395F69587957795A5
:102E30006795B795F111F8CFFAF4BB0F11F460FF65
:102E40001BC06F5F7F4F8F4F9F4F16C0882311F0BD
:102E500096E911C0772321F09EE8872F762F05C0D1
:102E6000662371F096E8862F70E060E02AF09A956C
:102E7000660F771F881FDAF7880F9695879597F961
:102E80000895990F0008550FAA0BE0E8FEEF1616FB
:102E90001706E807F907C0F012161306E407F5074E
:102EA00098F0621B730B840B950B39F40A2661F0C2
:102EB000232B242B252B21F408950A2609F4A14065
:102EC000A6958FEF811D811D089597F99F6780E872
:102ED00070E060E008959FEF80EC089500240A946C
:102EE0001616170618060906089500240A941216E5
:102EF0001306140605060895092E0394000C11F418
:102F0000882352F0BB0F40F4BF2B11F460FF04C0C4
:102F10006F5F7F4F8F4F9F4F089557FD9058440F1D
:102F2000551F59F05F3F71F04795880F97FB991F28
:102F300061F09F3F79F087950895121613061406E5
:102F4000551FF2CF4695F1DF08C016161706180672
:102F5000991FF1CF86957105610508940895E8944D
:102F6000BB2766277727CB0197F908958ADF08F4F6
:102F70008FEF08950BD0C0CFB1DF28F0B6DF18F087
:102F8000952309F0A2CFA7CF1124EACFC6DFA0F383
:102F9000959FD1F3950F50E0551F629FF001729FEE
:102FA000BB27F00DB11D639FAA27F00DB11DAA1F0D
:102FB000649F6627B00DA11D661F829F2227B00D5A
:102FC000A11D621F739FB00DA11D621F839FA00DE5
:102FD000611D221F749F3327A00D611D231F849F35
:102FE000600D211D822F762F6A2F11249F5750408C
:102FF0008AF0E1F088234AF0EE0FFF1FBB1F661F27
:10300000771F881F91505040A9F79E3F510570F0DF
:103010005CCFA6CF5F3FECF3983EDCF386957795C7
:103020006795B795F795E7959F5FC1F7FE2B880FDA
:10303000911D9695879597F9089597FB092E072678
:103040000AD077FD04D049D006D000201AF470953C
:1030500061957F4F0895F6F7909581959F4F08955C
:10306000A1E21A2EAA1BBB1BFD010DC0AA1FBB1F8C
:10307000EE1FFF1FA217B307E407F50720F0A21BFE
:10308000B30BE40BF50B661F771F881F991F1A946B
:1030900069F760957095809590959B01AC01BD0195
:1030A000CF01089597FB092E05260ED057FD04D0B9
:1030B000D7DF0AD0001C38F4509540953095219503
:1030C0003F4F4F4F5F4F0895F6F79095809570955D
:1030D00061957F4F8F4F9F4F0895AA1BBB1B51E1F6
:1030E00007C0AA1FBB1FA617B70710F0A61BB70B78
:1030F000881F991F5A95A9F780959095BC01CD011D
:103100000895EE0FFF1F0590F491E02D09949111A1
:1031100006C0803219F089508550D0F7089599275C
:10312000882708952F923F924F925F926F927F92DD
:103130008F929F92AF92BF92CF92DF92EF92FF92C7
:103140000F931F93CF93DF93CDB7DEB7CA1BDB0B73
:103150000FB6F894DEBF0FBECDBF09942A88398818
:1031600048885F846E847D848C849B84AA84B9841F
:10317000C884DF80EE80FD800C811B81AA81B9812B
:10318000CE0FD11D0FB6F894DEBF0FBECDBFED013F
:10319000089511E0C2E0D1E004C0FE010E9483184E
:0C31A0002296C430D107C9F7F894FFCF85
:1031AC00007B22736F667477617265223A222573F5
:1031BC00222C2022706F776572223A25622C2022F5
:1031CC006C656E677468223A25692C2022776964D5
:1031DC007468223A256900506C6F7474576172657B
:1031EC004669726D776172652076302E302E310013
:1031FC00583A256620593A25660050524F4752419D
:10320C004D20454E44004F4B0020003B0028002928
:10321C000047300047310047340047323800473907
:10322C0030004739310054004D313132004D3131CD
:10323C0034004D313135004D31313800436F6D6DF7
:10324C00616E64206E6F7420737570706F7274652C
:10325C00642E004D320050656E310050656E3200A8
:10326C0050656E33000000200005030000FFFFFFD7
:10327C00FFFFFFFFFFFFFFFFFFFFFFFFFF0000004F
:0E328C00000611AB119C10CD10AD10F6100015
:00000001FF
